** EXPERIMENTAL (HLL) ** Open Watcom Linker Version 1.6beta1 Limited Availability
Portions Copyright (c) 1985-2002 Sybase, Inc. All Rights Reserved.
Created on:       13/11/17 16:25:25
Warning! W1121: file U:/tmp\ldconv__cursesmodule_obj_1a7352885a4c11f40.obj(U:\DEV\python-2.7.5\Modules\_cursesmodule.c): '_init_curses' has already been exported
Executable Image: build/lib.os2knix-2.7/_curses.pyd
creating an OS/2 EMX dynamic link library


                        +------------+
                        |   Groups   |
                        +------------+

Group                           Address              Size
=====                           =======              ====

CGROUP                          0001:00000000        00037960
DGROUP                          0002:00000000        00001cd0



                        +--------------+
                        |   Segments   |
                        +--------------+

Segment                Class          Group          Address         Size
=======                =====          =====          =======         ====

TEXT32                 CODE           CGROUP         0001:00000000   00037960
________TEXT           CODE           CGROUP         0001:00037960   00000000
DATA32                 DATA           DGROUP         0002:00000000   00001210
SET1__os2dll           DATA           DGROUP         0002:00001210   00000004
SET2__os2dll           DATA           DGROUP         0002:00001214   00000000
SET3__os2dll           DATA           DGROUP         0002:00001214   00000004
SET1___CTOR_LIST__     DATA           DGROUP         0002:00001218   00000004
SET2___CTOR_LIST__     DATA           DGROUP         0002:0000121c   00000000
SET3___CTOR_LIST__     DATA           DGROUP         0002:0000121c   00000004
SET1___DTOR_LIST__     DATA           DGROUP         0002:00001220   00000004
SET2___DTOR_LIST__     DATA           DGROUP         0002:00001224   00000000
SET3___DTOR_LIST__     DATA           DGROUP         0002:00001224   00000004
SET1___crtinit1__      DATA           DGROUP         0002:00001228   00000004
SET2___crtinit1__      DATA           DGROUP         0002:0000122c   00000000
SET3___crtinit1__      DATA           DGROUP         0002:0000122c   00000004
SET1___crtexit1__      DATA           DGROUP         0002:00001230   00000004
SET2___crtexit1__      DATA           DGROUP         0002:00001234   00000000
SET3___crtexit1__      DATA           DGROUP         0002:00001234   00000004
SET1___eh_frame__      DATA           DGROUP         0002:00001238   00000004
SET2___eh_frame__      DATA           DGROUP         0002:0000123c   00000008
SET3___eh_frame__      DATA           DGROUP         0002:00001244   00000004
SET1___eh_init__       DATA           DGROUP         0002:00001248   00000004
SET2___eh_init__       DATA           DGROUP         0002:0000124c   00000004
SET3___eh_init__       DATA           DGROUP         0002:00001250   00000004
SET1___eh_term__       DATA           DGROUP         0002:00001254   00000004
SET2___eh_term__       DATA           DGROUP         0002:00001258   00000004
SET3___eh_term__       DATA           DGROUP         0002:0000125c   00000004
SET1___fork_parent1__  DATA           DGROUP         0002:00001260   00000004
SET2___fork_parent1__  DATA           DGROUP         0002:00001264   00000000
SET3___fork_parent1__  DATA           DGROUP         0002:00001264   00000004
SET1___fork_child1__   DATA           DGROUP         0002:00001268   00000004
SET2___fork_child1__   DATA           DGROUP         0002:0000126c   00000000
SET3___fork_child1__   DATA           DGROUP         0002:0000126c   00000004
________DATA           DATA           DGROUP         0002:00001270   00000000
BSS32                  BSS            DGROUP         0002:00001270   00000a60
c_common               BSS            DGROUP         0002:00001cd0   00000000
________BSS            BSS            DGROUP         0002:00001cd0   00000000


                        +----------------+
                        |   Memory Map   |
                        +----------------+

* = unreferenced symbol
+ = symbol only referenced locally

Address        Symbol
=======        ======

Module: U:\usr\lib\dll0hi.obj({standard input})
0001:00000000* __text
0002:00000000* __data
0002:00000000* ___data_start
0002:00001270* ___bss_start
0002:00001210+ __os2dll
0002:00001218  ___CTOR_LIST__
0002:00001220  ___DTOR_LIST__
0002:00001228* ___crtinit1__
0002:00001230* ___crtexit1__
0002:00001238  ___eh_frame__
0002:00001248  ___eh_init__
0002:00001254  ___eh_term__
0002:00001260+ ___fork_parent1__
0002:00001268+ ___fork_child1__
Module: U:/tmp\ldconv__cursesmodule_obj_1a7352885a4c11f40.obj(U:\DEV\python-2.7.5\Modules\_cursesmodule.c)
0001:000084c7  _init_curses
0002:00000050* _PyCursesWindow_Type
0002:00000114* _PyCursesVersion
Module: U:\usr\local473\lib\libc_dll.lib(dllinit.obj)
0001:000099d0  _DLL_InitTerm
Module: U:\usr\lib\libend.lib(src/libend/386/endlink386.asm)
0002:00001cd0  _end
0002:00001270  _edata
Module: U:\usr\lib\libend.lib(src/libend/386/end.asm)
0001:00037960* _etext
0001:00037960* __etext
0000:00000000* WEAK$ZERO
0002:00001cd0  __end
0002:00001270  __edata
Module: U:\extras\lib\ncurses.lib(lib_options.obj)
0001:00009a30  _curs_set
0001:00009af0  _idlok
0001:00009b50  _idcok
0001:00009ba0  _halfdelay
0001:00009bf0  _nodelay
0001:00009c20  _notimeout
0001:00009c40  _wtimeout
0001:00009c60  _keypad
0001:00009cf0  _meta
0001:00009d60  _typeahead
0001:00009d80  _has_key
0001:00009e00  __nc_keypad
Module: U:\extras\lib\ncurses.lib(lib_window.obj)
0001:00009ef0  _wsyncup
0001:00009fc0  _wsyncdown
0001:0000a0a0  _dupwin
0001:0000a2b0  __nc_synchook
0001:0000a2f0  _mvderwin
0001:0000a410  _syncok
0001:0000a430  _wcursyncup
Module: U:\extras\lib\ncurses.lib(lib_move.obj)
0001:0000a490  _wmove
Module: U:\extras\lib\ncurses.lib(lib_instr.obj)
0001:0000a4e0  _winnstr
Module: U:\extras\lib\ncurses.lib(lib_winch.obj)
0001:0000a570  _winch
Module: U:\extras\lib\ncurses.lib(lib_immedok.obj)
0001:0000a5a0  _immedok
Module: U:\extras\lib\ncurses.lib(lib_getstr.obj)
0001:0000a5c0  _wgetnstr
Module: U:\extras\lib\ncurses.lib(lib_getch.obj)
0001:0000aaa0* __nc_wgetch
0001:0000b300  _wgetch
0002:00000a70  _ESCDELAY
Module: U:\extras\lib\ncurses.lib(lib_keyname.obj)
0001:0000ba60* __nc_key_names
0001:0000bf50  _keyname
Module: U:\extras\lib\ncurses.lib(lib_mouse.obj)
0001:0000c570* _wmouse_trafo
0001:0000c6a0  _getmouse
0001:0000c720  _ungetmouse
0001:0000c790  _mousemask
0001:0000c880  _wenclose
0001:0000c900  _mouseinterval
0001:0000c930* __nc_has_mouse
Module: U:\extras\lib\ncurses.lib(lib_clreol.obj)
0001:0000d5e0  _wclrtoeol
Module: U:\extras\lib\ncurses.lib(lib_clrbot.obj)
0001:0000d6b0  _wclrtobot
Module: U:\extras\lib\ncurses.lib(lib_clear.obj)
0001:0000d780  _wclear
Module: U:\extras\lib\ncurses.lib(lib_box.obj)
0001:0000d7b0  _wborder
Module: U:\extras\lib\ncurses.lib(lib_data.obj)
0002:000012e0  _stdscr
0002:000012e4  _curscr
0002:000012e8  _newscr
0002:000012ec  __nc_screen_chain
0002:000012f0  _SP
Module: U:\extras\lib\ncurses.lib(lib_delwin.obj)
0001:0000d9a0  _delwin
Module: U:\extras\lib\ncurses.lib(lib_tparm.obj)
0001:0000da70* __nc_tparm_analyze
0001:0000dda0  _tparm
0002:00001300* __nc_tparm_err
Module: U:\extras\lib\ncurses.lib(lib_color.obj)
0001:0000f080  _start_color
0001:0000f310  _init_pair
0001:0000f620  __nc_do_color
0001:0000f9a0  __nc_reset_colors
0001:0000fa30  _init_color
0001:0000fd10  _can_change_color
0001:0000fd30  _has_colors
0001:0000fdb0  _color_content
0001:0000fe50  _pair_content
0002:000014f0  _COLOR_PAIRS
0002:000014f4  _COLORS
Module: U:\extras\lib\ncurses.lib(lib_setup.obj)
0001:000101b0* __nc_setupterm
0001:00010650  _use_env
0001:00010660* __nc_get_locale
0001:00010690  __nc_unicode_locale
0001:00010700  __nc_locale_breaks_acs
0001:00010860  _setupterm
0002:00000aa0  _ttytype
0002:00001500  _LINES
0002:00001504  _COLS
0002:00001508  _TABSIZE
Module: U:\extras\lib\ncurses.lib(lib_kernel.obj)
0001:000109c0  _erasechar
0001:000109f0  _killchar
0001:00010a20  _flushinp
Module: U:\extras\lib\ncurses.lib(lib_newterm.obj)
0001:00010a90  _newterm
0001:00010d80  _filter
0001:00010d90* _nofilter
Module: U:\extras\lib\ncurses.lib(lib_touch.obj)
0001:00010da0  _is_linetouched
0001:00010de0  _is_wintouched
0001:00010e20  _wtouchln
Module: U:\extras\lib\ncurses.lib(lib_dft_fgbg.obj)
0001:00010ef0  _use_default_colors
0001:00010fc0* _assume_default_colors
Module: U:\extras\lib\ncurses.lib(unctrl.obj)
0001:000117f0  _unctrl
Module: U:\extras\lib\ncurses.lib(lib_ti.obj)
0001:00011850  _tigetflag
0001:000118c0  _tigetnum
0001:00011940  _tigetstr
Module: U:\extras\lib\ncurses.lib(lib_termname.obj)
0001:000119c0  _termname
Module: U:\extras\lib\ncurses.lib(lib_vidattr.obj)
0001:000119e0* _vidputs
0001:000122e0  _vidattr
0001:00012300  _termattrs
Module: U:\extras\lib\ncurses.lib(lib_raw.obj)
0001:000123b0  _raw
0001:00012470  _cbreak
0001:00012520  _qiflush
0001:00012580  _noraw
0001:00012640  _nocbreak
0001:000126e0  _noqiflush
0001:00012740  _intrflush
Module: U:\extras\lib\ncurses.lib(lib_napms.obj)
0001:000127c0  _napms
Module: U:\extras\lib\ncurses.lib(lib_longname.obj)
0001:00012830  _longname
Module: U:\extras\lib\ncurses.lib(resizeterm.obj)
0001:00012880  _resize_term
0001:00012d90  _is_term_resized
0001:00012de0  _resizeterm
Module: U:\extras\lib\ncurses.lib(lib_isendwin.obj)
0001:00012e90  _isendwin
Module: U:\extras\lib\ncurses.lib(lib_has_cap.obj)
0001:00012eb0  _has_ic
0001:00012f20  _has_il
Module: U:\extras\lib\ncurses.lib(lib_baudrate.obj)
0001:00012ff0  __nc_baudrate
0001:00013040  __nc_ospeed
0001:00013080  _baudrate
Module: U:\extras\lib\ncurses.lib(lib_insdel.obj)
0001:000130d0  _winsdelln
Module: U:\extras\lib\ncurses.lib(lib_erase.obj)
0001:00013130  _werase
Module: U:\extras\lib\ncurses.lib(lib_redrawln.obj)
0001:000131f0  _wredrawln
Module: U:\extras\lib\ncurses.lib(lib_clearok.obj)
0001:00013320  _clearok
Module: U:\extras\lib\ncurses.lib(lib_wattron.obj)
0001:00013340  _wattr_on
Module: U:\extras\lib\ncurses.lib(lib_wattroff.obj)
0001:00013380  _wattr_off
Module: U:\extras\lib\ncurses.lib(lib_mvwin.obj)
0001:000133b0  _mvwin
Module: U:\extras\lib\ncurses.lib(lib_leaveok.obj)
0001:00013450  _leaveok
Module: U:\extras\lib\ncurses.lib(wresize.obj)
0001:00013560  _wresize
Module: U:\extras\lib\ncurses.lib(lib_scrreg.obj)
0001:00013940  _wsetscrreg
Module: U:\extras\lib\ncurses.lib(lib_scrollok.obj)
0001:00013990  _scrollok
Module: U:\extras\lib\ncurses.lib(lib_tputs.obj)
0001:00013e10  __nc_outch
0001:000139b0  _tputs
0001:00013d10  _delay_output
0001:00013de0  __nc_flush
0001:00013e70  _putp
0002:00001570  _PC
0002:00001572  _ospeed
0002:00001574* __nc_nulls_sent
Module: U:\extras\lib\ncurses.lib(lib_screen.obj)
0001:00013ea0  _getwin
0001:00014080  _putwin
0001:00014150* _scr_restore
0001:000141d0* _scr_dump
0001:00014240* _scr_init
0001:000142e0* _scr_set
Module: U:\extras\lib\ncurses.lib(lib_addstr.obj)
0001:000143c0* _waddchnstr
0001:000144d0  _waddnstr
Module: U:\extras\lib\ncurses.lib(lib_insnstr.obj)
0001:00014560  _winsnstr
Module: U:\extras\lib\ncurses.lib(lib_chgat.obj)
0001:000145f0  _wchgat
Module: U:\extras\lib\ncurses.lib(lib_nl.obj)
0001:00014700  _nl
0001:00014750  _nonl
Module: U:\extras\lib\ncurses.lib(lib_echo.obj)
0001:000147a0  _echo
0001:000147c0  _noecho
Module: U:\extras\lib\ncurses.lib(lib_ttyflags.obj)
0001:000147e0  __nc_get_tty_mode
0001:00014860  __nc_set_tty_mode
0001:000148e0  _def_shell_mode
0001:00014960  _def_prog_mode
0001:000149e0  _reset_prog_mode
0001:00014a90  _reset_shell_mode
0001:00014b60  _savetty
0001:00014be0  _resetty
Module: U:\extras\lib\ncurses.lib(lib_endwin.obj)
0001:00014c60  _endwin
Module: U:\extras\lib\ncurses.lib(lib_flash.obj)
0001:00014ca0  _flash
Module: U:\extras\lib\ncurses.lib(lib_beep.obj)
0001:00014cf0  _beep
Module: U:\extras\lib\ncurses.lib(tty_update.obj)
0001:00014d60  _doupdate
0001:00017180* __nc_screen_resume
0001:00016ad0  __nc_scrolln
0001:00017320  __nc_screen_init
0001:00017330  __nc_screen_wrap
Module: U:\extras\lib\ncurses.lib(lib_delch.obj)
0001:00019550  _wdelch
Module: U:\extras\lib\ncurses.lib(lib_ungetch.obj)
0001:00019610  _ungetch
Module: U:\extras\lib\ncurses.lib(lib_refresh.obj)
0001:000196e0  _wnoutrefresh
0001:000198f0  _wrefresh
Module: U:\extras\lib\ncurses.lib(lib_pad.obj)
0001:00019960  _pnoutrefresh
0001:00019c80  _newpad
0001:00019d50  _subpad
0001:00019da0  _prefresh
0001:00019e00  _pechochar
Module: U:\extras\lib\ncurses.lib(lib_initscr.obj)
0001:00019ec0  _initscr
Module: U:\extras\lib\ncurses.lib(lib_acs.obj)
0001:00019f60  __nc_init_acs
0002:000015c0  _acs_map
Module: U:\extras\lib\ncurses.lib(lib_scroll.obj)
0001:0001a2e0  __nc_scroll_window
0001:0001a540  _wscrl
Module: U:\extras\lib\ncurses.lib(lib_newwin.obj)
0001:0001a5a0  __nc_freewin
0001:0001a670  __nc_makenew
0001:0001a8c0  _newwin
0001:0001a9d0  _derwin
0001:0001ab10  _subwin
Module: U:\extras\lib\ncurses.lib(lib_insch.obj)
0001:0001ad10  __nc_insert_ch
0001:0001af20  _winsch
Module: U:\extras\lib\ncurses.lib(lib_addch.obj)
0001:0001af90  __nc_render
0001:0001b050  __nc_waddch_nosync
0001:0001b060  _waddch
0001:0001b0b0  _wechochar
Module: U:\extras\lib\ncurses.lib(lib_bkgd.obj)
0001:0001b8b0  _wbkgdset
0001:0001b8c0  _wbkgd
Module: U:\extras\lib\ncurses.lib(lib_hline.obj)
0001:0001ba70  _whline
Module: U:\extras\lib\ncurses.lib(lib_vline.obj)
0001:0001bb30  _wvline
Module: U:\extras\lib\ncurses.lib(lib_overlay.obj)
0001:0001bc00  _copywin
0001:0001bdc0  _overlay
0001:0001bdf0  _overwrite
Module: U:\tmp\ldconv_libgcc_so_d_a_1a7352885a4c1d32e8.lib(emx-ctordtor.obj)
0001:0001bf30  ___ctordtorInit
0001:0001bf64  ___ctordtorTerm
Module: U:\extras\lib\ncurses.lib(lib_cur_term.obj)
0001:0001bfa0  _set_curterm
0001:0001c000  _del_curterm
0002:000017d0  _cur_term
Module: U:\extras\lib\ncurses.lib(init_keytry.obj)
0001:0001c060  __nc_init_keytry
0002:00000c50* __nc_tinfo_fkeys
Module: U:\extras\lib\ncurses.lib(lib_twait.obj)
0001:0001c1a0  __nc_timed_wait
Module: U:\extras\lib\ncurses.lib(lib_trace.obj)
0002:000018f0  __nc_tracing
Module: U:\extras\lib\ncurses.lib(keybound.obj)
0001:0001c3d0  _keybound
Module: U:\extras\lib\ncurses.lib(names.obj)
0001:0001c4e0  _boolnames
0001:0001c880  _boolfnames
0001:0001ca00  _numnames
0001:0001cd00  _numfnames
0001:0001d580  _strnames
0001:0001efc0  _strfnames
Module: U:\extras\lib\ncurses.lib(add_tries.obj)
0001:0001f640  __nc_add_to_try
Module: U:\extras\lib\ncurses.lib(keyok.obj)
0001:0001f7d0  _keyok
Module: U:\usr\lib\libos2.lib(mou17.obj)
0001:0001f8f0  MouOpen
Module: U:\usr\lib\libos2.lib(mou16.obj)
0001:0001f940  MouSetEventMask
Module: U:\usr\lib\libos2.lib(mou26.obj)
0001:0001f990  MouDrawPtr
Module: U:\usr\lib\libos2.lib(mou20.obj)
0001:0001f9c0  MouReadEventQue
Module: U:\usr\lib\libos2.lib(mou9.obj)
0001:0001fa10  MouClose
Module: U:\extras\lib\ncurses.lib(doalloc.obj)
0001:0001fa40  __nc_doalloc
Module: U:\extras\lib\ncurses.lib(comp_error.obj)
0001:0001fad0  __nc_warning
0001:0001fbe0  __nc_err_abort
0001:0001fcf0  __nc_syserr_abort
0001:0001fe00* __nc_get_source
0001:0001fe10* __nc_set_source
0001:0001fe20  __nc_set_type
0001:0001fe80  __nc_get_type
0002:00001910  __nc_suppress_warnings
0002:00001914  __nc_curr_line
0002:00001918  __nc_curr_col
Module: U:\extras\lib\ncurses.lib(hashmap.obj)
0001:0001fec0  __nc_hash_map
0001:000203f0  __nc_make_oldhash
0001:00020450  __nc_scroll_oldhash
Module: U:\extras\lib\ncurses.lib(read_entry.obj)
0001:00020dd0* __nc_read_termtype
0001:00021830* __nc_read_file_entry
0001:000218e0  __nc_read_entry
Module: U:\extras\lib\ncurses.lib(fallback.obj)
0001:00021bb0  __nc_fallback
Module: U:\extras\lib\ncurses.lib(name_match.obj)
0001:00021bc0  __nc_name_match
0001:00021cb0  __nc_first_name
Module: U:\extras\lib\ncurses.lib(getenv_num.obj)
0001:00021d20  __nc_getenv_num
Module: U:\extras\lib\ncurses.lib(lib_slk.obj)
0001:00021d90  __nc_slk_initialize
0001:00022320* _slk_restore
0002:00001950  __nc_slk_format
Module: U:\extras\lib\ncurses.lib(lib_set_term.obj)
0001:00022440* _delscreen
0001:00022740  __nc_setupscreen
0001:00022de0* __nc_ripoffline
0001:00022e20  _set_term
0001:00022e90* _ripoffline
Module: U:\extras\lib\ncurses.lib(lib_mvcur.obj)
0001:00022f60* __nc_msec_cost
0001:000230e0  __nc_mvcur_init
0001:00023ac0  _mvcur
0001:00023cb0  __nc_mvcur_resume
0001:00023d60  __nc_mvcur_wrap
Module: U:\extras\lib\ncurses.lib(lib_tstp.obj)
0001:00024c10  __nc_signal_handler
Module: U:\extras\lib\ncurses.lib(access.obj)
0001:000250c0* __nc_rootname
0001:00025160* __nc_is_abs_path
0001:000251a0  __nc_pathlast
0001:000251f0* __nc_basename
0001:00025240  __nc_access
0001:00025310  __nc_is_dir_path
0001:00025360* __nc_is_file_path
Module: U:\extras\lib\ncurses.lib(setbuf.obj)
0001:000253d0  __nc_set_buffer
Module: U:\extras\lib\ncurses.lib(hardscroll.obj)
0001:00025490  __nc_scroll_optimize
0002:00001a00  __nc_oldnums
Module: U:\tmp\ldconv_libgcc_so_d_a_1a7352885a4c1d32e8.lib(emx-eh.obj)
0001:00025660  ___ehInit
0001:00025696* ___ehTerm
Module: U:\extras\lib\ncurses.lib(free_ttype.obj)
0001:000256d0  __nc_free_termtype
0001:00025790* _use_extended_names
0002:00001190  __nc_user_definable
Module: U:\extras\lib\ncurses.lib(key_defined.obj)
0001:00025840  _key_defined
Module: U:\extras\lib\ncurses.lib(tries.obj)
0001:00025880  __nc_expand_try
0001:00025940  __nc_remove_key
0001:000259c0* __nc_remove_string
Module: U:\tmp\ldconv_libgcc_a_1a7352885a4c1afc8.lib(_alloca.obj)
0001:00025a20  __alloca
Module: U:\extras\lib\ncurses.lib(db_iterator.obj)
0001:00025aa0  __nc_next_db
0001:00025be0* __nc_tic_dir
0001:00025c30* __nc_keep_tic_dir
0001:00025c80  __nc_last_db
0001:00025cc0* __nc_first_db
Module: U:\extras\lib\ncurses.lib(lib_printw.obj)
0001:00025db0* _printw
0001:00025eb0* _vwprintw
0001:00025de0* _wprintw
0001:00025e10* _mvprintw
0001:00025e60  _mvwprintw
Module: U:\extras\lib\ncurses.lib(lib_slkrefr.obj)
0001:00025f00* _slk_noutrefresh
0001:00025f60  _slk_refresh
Module: U:\extras\lib\ncurses.lib(strings.obj)
0001:00026190  __nc_str_init
0001:000261c0  __nc_str_null
0001:000261f0  __nc_str_copy
0001:00026220  __nc_safe_strcat
0001:00026290  __nc_safe_strcpy
Module: U:\extras\lib\ncurses.lib(comp_parse.obj)
0001:00026300* __nc_delink_entry
0001:000263b0* __nc_read_entry_source
0001:000265a0* __nc_resolve_uses2
0001:00027ea0* __nc_free_entries
0001:00027ed0  __nc_free_entry
0001:00027f00* __nc_entry_match
0001:000280a0* __nc_resolve_uses
0002:000011c0* __nc_check_termtype2
0002:000011c4* __nc_check_termtype
0002:00001a70  __nc_head
0002:00001a74* __nc_tail
Module: U:\extras\lib\ncurses.lib(home_terminfo.obj)
0001:00028100  __nc_home_terminfo
Module: U:\extras\lib\ncurses.lib(safe_sprintf.obj)
0001:00028190  __nc_printf_string
Module: U:\extras\lib\ncurses.lib(comp_scan.obj)
0001:00028530  __nc_get_token
0001:00029330  __nc_panic_mode
0001:00028e50* __nc_trans_string
0001:00029350  __nc_reset_input
0001:000293b0  __nc_push_token
0002:00001ad0  __nc_syntax
0002:00001ad4* __nc_curr_file_pos
0002:00001ad8  __nc_comment_start
0002:00001adc  __nc_comment_end
0002:00001ae0  __nc_start_line
0002:00001ae4  __nc_curr_token
0002:00001af0* __nc_disable_period
Module: U:\extras\lib\ncurses.lib(parse_entry.obj)
0001:0002a0a0  __nc_parse_entry
0001:0002a830* __nc_capcmp
Module: U:\extras\lib\ncurses.lib(alloc_entry.obj)
0001:0002c010  __nc_wrap_entry
0001:0002c580  __nc_merge_entry
0001:0002c680  __nc_init_entry
0001:0002c7a0  __nc_copy_entry
0001:0002c810  __nc_save_str
Module: U:\extras\lib\ncurses.lib(alloc_ttype.obj)
0001:0002c8b0  __nc_align_termtype
0001:0002cb90  __nc_copy_termtype
Module: U:\extras\lib\ncurses.lib(comp_captab.obj)
0001:0002f910  __nc_info_hash_table
0001:00032550  __nc_cap_hash_table
0001:00033570  __nc_capalias_table
0001:000337b0  __nc_infoalias_table
0001:00033810  __nc_get_table
0001:00033830* __nc_get_hash_table
Module: U:\extras\lib\ncurses.lib(comp_hash.obj)
0001:00033850  __nc_find_entry
0001:000338f0  __nc_find_type_entry
Module: U:\extras\lib\ncurses.lib(captoinfo.obj)
0001:00033a30  __nc_captoinfo
0001:00034ce0* __nc_infotocap
Module: U:\extras\lib\ncurses.lib(visbuf.obj)
0001:000376d0* __nc_visbuf2
0001:00037770  __nc_visbuf
0001:00037790* __nc_visbufn


                        +----------------------+
                        |   Imported Symbols   |
                        +----------------------+

Symbol                              Module
======                              ======

___libc_ForkRegisterModule          libc065
___init_dll                         libc065
___libc_Back_termDll                libc065
___libc_ForkDeregisterModule        libc065
__atfork_callback                   libc065
__Py_NoneStruct                     python27
_Py_FindMethod                      python27
_PyArg_ParseTuple                   python27
_PyTuple_Size                       python27
_PyExc_TypeError                    python27
_PyErr_SetString                    python27
_PyString_FromString                python27
_PyInt_FromLong                     python27
_Py_BuildValue                      python27
_PyEval_SaveThread                  python27
_PyEval_RestoreThread               python27
_PyErr_CheckSignals                 python27
_PyErr_Occurred                     python27
_PyObject_Free                      python27
_PyDict_SetItemString               python27
_PyArg_ParseTupleAndKeywords        python27
_PySys_GetObject                    python27
_PyObject_AsFileDescriptor          python27
_PyImport_ImportModuleNoBlock       python27
_PyObject_SetAttrString             python27
_PyString_FromStringAndSize         python27
__Py_TrueStruct                     python27
__Py_ZeroStruct                     python27
_PyExc_ValueError                   python27
_PyString_AsString                  python27
_PyInt_AsLong                       python27
_PyErr_Format                       python27
_PyString_Size                      python27
_PyFile_Type                        python27
_PyType_IsSubtype                   python27
_PyFile_AsFile                      python27
_PyObject_Malloc                    python27
_PyObject_Init                      python27
_PyType_Type                        python27
_Py_InitModule4                     python27
_PyModule_GetDict                   python27
_PyCapsule_New                      python27
_PyErr_NewException                 python27
_PyErr_NoMemory                     python27
__CRT_init                          libc065
__CRT_term                          libc065
DosCreateThread                     doscalls
DosExit                             doscalls
DosWrite                            doscalls
___libc_GLocaleCtype                libc065
___stderrp                          libc065
__scrsize                           libc065
__errno                             libc065
___stdoutp                          libc065
__fsetmode                          libc065
___stdinp                           libc065
__std_malloc                        libc065
__std_free                          libc065
___ctordtorInit1                    libc065
___ctordtorTerm1                    libc065
__std_read                          libc065
__std_sprintf                       libc065
__std_strdup                        libc065
__std_calloc                        libc065
__std_strcmp                        libc065
__std_strstr                        libc065
__std_pipe                          libc065
__std_setmode                       libc065
__std_printf                        libc065
__std_getenv                        libc065
__std_strlen                        libc065
__std_perror                        libc065
__libc_32to16                       libc065
_16_Mou16Open                       moucalls
__libc_thunk1                       libc065
_16_Mou16SetEventMask               moucalls
_16_Mou16DrawPtr                    moucalls
_16_Mou16ReadEventQue               moucalls
__std_strncpy                       libc065
_16_Mou16Close                      moucalls
__std_fprintf                       libc065
__std_exit                          libc065
__std_isatty                        libc065
__std_fwrite                        libc065
__std_setlocale                     libc065
__std_nl_langinfo                   libc065
__std_atoi                          libc065
__std_strchr                        libc065
__std_tcflush                       libc065
__std_fileno                        libc065
__std_nanosleep                     libc065
__std_cfgetospeed                   libc065
__std_fflush                        libc065
__std_putc                          libc065
__std_write                         libc065
__std_clearerr                      libc065
__std_fread                         libc065
__std_fopen                         libc065
__std_fclose                        libc065
__std_tcgetattr                     libc065
__std_tcsetattr                     libc065
__std_select                        libc065
___register_frame_table             gcc473
___deregister_frame                 gcc473
__std_gettimeofday                  libc065
__std_realloc                       libc065
__std_fputc                         libc065
__std_vfprintf                      libc065
__std_strncat                       libc065
__std_strcpy                        libc065
__std_memmove                       libc065
__std_memcpy                        libc065
__std_memset                        libc065
__std_open                          libc065
__std_close                         libc065
__std_strtol                        libc065
__std_sscanf                        libc065
__std_sigaction                     libc065
__std_sigemptyset                   libc065
__std_sigaddset                     libc065
__std_sigprocmask                   libc065
__std_sigismember                   libc065
__std_getpid                        libc065
__std_kill                          libc065
__std_tcgetpgrp                     libc065
__std_getpgrp                       libc065
__std_strrchr                       libc065
__std_access                        libc065
__std_stat                          libc065
__std_setvbuf                       libc065
__std_vsnprintf                     libc065
__std_ftell                         libc065
__std_fgets                         libc065
__std_strcat                        libc065
__std_strncmp                       libc065


                        +--------------------+
                        |   Libraries Used   |
                        +--------------------+

U:\extras\lib\ncurses.lib
U:\tmp\ldconv_python2_7_dll_a_1a7352885a4c17530.lib
U:\tmp\ldconv_libgcc_a_1a7352885a4c1afc8.lib
U:\tmp\ldconv_libgcc_so_d_a_1a7352885a4c1d32e8.lib
U:\usr\lib\libc_alias.lib
U:\usr\local473\lib\libc_dll.lib
U:\usr\lib\libos2.lib
U:\usr\lib\libend.lib


                        +-----------------------+
                        |   Linker Statistics   |
                        +-----------------------+

Stack size:  0000 (0.)
Memory size:  00039630 (235056.)
Link time: 00:00.12
